:020000040000FA
:0400000068303A2802
:08000800A000030EA100831209
:1000100005191028831601178312B23081002B288E
:1000200083160113831203140B190310A80DA90DD5
:10003000AA0DAB0DAC0DAC16FF302C02031D2B2806
:10004000FA302B02031D2B2831152A08AF0029088E
:10005000AE002808AD008B100B11210E8300A00EFE
:04006000200E090065
:0C007400203084008001840A6030040207
:10008000031C3C281230B00052218316FF2390003D
:10009000831283160C308505870183128501870141
:1000A000073099000030831691009F008312C830FA
:1000B00083168100831231309000003083168C004B
:1000C000831210308B00831600309B001C141A081A
:1000D0008312BC00851D69213C1C762883161030D4
:1000E0009B001C141A088312BD005E2181018E0141
:1000F0008F010B118B100B108C018B178E20311977
:1001000091203621B30B8C28031085190314B90DE7
:10011000F03039020319E9208F217E286400321063
:10012000080031110130B7008B13203037078316D8
:100130009B001C141A088312A40010303707831682
:100140009B001C141A088312A300A6000230A60606
:100150000030370783169B001C141A088312A20074
:10016000A7000130A7068B17321CBC2822090339CF
:10017000A200A309A409A50924082F02031DE3284E
:1001800023082E02031DD12822082D02031DE32877
:1001900001303702031DD1283D18D1283D143E14EB
:1001A000532126082E02031DE32827082D02031DD4
:1001B000E32801303702031DE2283D1CE2283D10F0
:1001C0003E145621E328B70A02303702031808000C
:1001D00094280130B600B300B400B500B700850123
:1001E0008701B1138E20B30B052903108519031461
:1001F000B90DF030390203192C29B40B052901304F
:10020000370203195A219630B400311DF2283111FA
:10021000321C0F292D090339AD00AE09AF092F1C7F
:10022000F2288E018F010C1CF2280C102E1EF228D1
:100230008B1320303707BB002F08BA003F21103046
:100240003707BB002E08BA003F2100303707BB003C
:100250002D08BA003F218B1785018701B70AB60127
:1002600002303702031CF2285E2108003E1C080001
:100270003E101030BB003D08BA003F2108008B1330
:100280003A0883161C159A003B089B0055309D00C8
:10029000AA309D009C1464009C184B291C118312E9
:1002A0008B17080008000130BD00080087010530E9
:1002B000D40008000508333A8500080001303D02EB
:1002C0000319632908000130D40056150730D30004
:1002D0000800B601B301B4013C1C7129BC01BC1477
:1002E0007329BC013C143C08B600640077297829C6
:1002F00079297A297B293330B41B8500B41F850105
:10030000B30B7529B40B75290310B60CB608031D81
:1003100075290030BB003C08BA003F2108008F0857
:10032000031908008E018F01D0080319DF29D00FAF
:10033000AC2956180516D618851656190514D6195F
:100340008514D60158180512D818851258190510A9
:10035000D8198510D801DF295008D1005618051684
:10036000D618851656190514D619851451080E028B
:100370000318C62958180512D818851258190510DF
:10038000D8198510FF305002031908008F08031D8B
:1003900008008E2051080E02031CC62956180512AB
:1003A000D618851256190510D61985105818051635
:1003B000D818851658190514D81985140800003066
:1003C0005302031DF8293D18F029051A581401306D
:1003D000051AD000851AD8140130851AD0000800FB
:1003E0000130D40056140130D0000130D300080091
:1003F000051AFE295614851AD814002AD614581442
:100400000130D000D40B080001305302031D122A22
:10041000D6150530D4000230D3003D180800D601AF
:10042000D301080002305302031D242A56158714F5
:10043000D8150330D4000330D3003D1808008701DD
:10044000D601D301D815080003305302031D342A06
:10045000871407150330D4000430D3003D1808007A
:100460008701D3015815080004305302031D452AA3
:100470008714071507140330D4000530D3003D1846
:1004800008008701D3015815080005305302031DE9
:10049000572A87140715071487160330D40006302F
:1004A000D3003D1808008701D30158150800063015
:1004B0005302031D6A2A87140715071487160716A7
:1004C0000330D4000730D3003D1808008701D30162
:1004D0005815080007305302031D7E2A871407159C
:1004E00007148716071687150130D4000730D3008C
:1004F0003D1808008701D301581508000030D300CB
:020500000800F1
:084000000700030004000800A2
:02400E00CC01E3
:10420000010078007A007C007E007B0079007F004E
:104210007D007A0078007E007C00FF00FF00FF0038
:104220000000F200F600FA00FE00F200F600FA00CC
:10423000FE00F200F600FA00FE00FF00FF00FF00A3
:10424000010005000500050005000900090009003E
:1042500009000D000D000D000D00FF00FF00FF0024
:10426000FF00FF00FF00FF00FF00FF00FF00FF0056
:10427000FF00FF00FF00FF00FF00FF00FF00FF0046
:10428000FF00FF00FF00FF00FF00FF00FF00FF0036
:10429000FF00FF00FF00FF00FF00FF00FF00FF0026
:1042A000FF00FF00FF00FF00FF00FF00FF00FF0016
:1042B000FF00FF00FF00FF00FF00FF00FF00FF0006
:1042C000FF00FF00FF00FF00FF00FF00FF00FF00F6
:1042D000FF00FF00FF00FF00FF00FF00FF00FF00E6
:1042E000FF00FF00FF00FF00FF00FF00FF00FF00D6
:1042F000FF00FF00FF00FF00FF00FF00FF00DD00E8
:00000001FF
